:020000040000FA
:100000005F2FFF30A600A700A800F830A900112735
:100010000030A600A700A8001830A9001127FF3063
:10002000A600A700A800F830A90011270030A600FC
:10003000A700A8001830A90011270030A60008303A
:10004000A7000030A8001830A90011270030A60032
:10005000A700A8001830A90011270030A60008301A
:10006000A7000030A8001830A90011270030A60012
:10007000A700A8001830A900112708002430A60006
:10008000A700A800F830A90011270030A600A7009B
:10009000A8001830A90011274930A600A700A80021
:1000A0001830A90011270030A600A700A8001830BA
:1000B000A90011279230A600A700A8001830A900B7
:1000C00011270030A600A700A8001830A9001127AA
:1000D0000330A600A700A800F830A90011270030BF
:1000E000A600A700A8001830A90011271C30A60000
:1000F000A700A8001830A90011270030A600A7000B
:10010000A8001830A9001127E030A600A700A80019
:100110001830A90011270030A600A700A800183049
:10012000A90011279230A600A700A8001830A90046
:1001300011270030A600A700A8001830A900112739
:100140004930A600A700A8001830A90011270030E8
:10015000A600A700A8001830A90011272430A60087
:10016000A700A800F830A90011270030A600A700BA
:10017000A8001830A9001127E030A600A700A800A9
:100180001830A90011270030A600A700A8001830D9
:10019000A90011271C30A600A700A8001830A9004C
:1001A00011270030A600A700A8001830A9001127C9
:1001B0000330A600A700A800F830A90011270030DE
:1001C000A600A700A8001830A90011270800FF30DA
:1001D000A6000030A700A8008030A9001127003039
:1001E000A600A700A800A90011270030A600FF3034
:1001F000A7000030A8004030A90011270030A60059
:10020000A700A800A90011270030A600A700FF3012
:10021000A8002030A90011270030A600A700A800E0
:10022000A90011270030A600FF30A7000030A80069
:100230004830A90011270030A600A700A800083008
:10024000A9001127FF30A6000030A700A8009030B9
:10025000A90011270030A600A700A8001030A900AF
:1002600011270030A600FF30A7000030A800503052
:10027000A90011270030A600A700A8001030A9008F
:1002800011270030A600A700FF30A8003830A900D1
:1002900011270030A600A700A8001830A9001127D8
:1002A0000030A600FF30A7000030A8005830A90099
:1002B00011270030A600A700A8001830A9001127B8
:1002C000FF30A6000030A700A8009030A900112739
:1002D0000030A600A700A8001030A90011270030A8
:1002E000A600FF30A7000030A8005030A900112759
:1002F0000030A600A700A8001030A9001127003088
:10030000A600A700FF30A8002830A9001127003060
:10031000A600A700A8000830A90011270030A600F9
:10032000FF30A7000030A8004830A9001127003096
:10033000A600A700A8000830A90011270800003077
:10034000A600A7002030A8001830A900112700300F
:10035000A600A7006030A8001830A90011270030BF
:10036000A600A700E030A8001830A900112700302F
:10037000A600A700F030A8001830A900112700300F
:10038000A600A700F230A8001830A90011270030FD
:10039000A600A700F330A8001830A90011270030EC
:1003A000A600A700F330A8003830A90011270030BC
:1003B000A600A700F730A8003830A90011270030A8
:1003C000A600A700FF30A8003830A9001127003090
:1003D000A6002030A700FF30A8003830A900112760
:1003E0000030A6006030A700FF30A8003830A90018
:1003F00011270030A600E030A700FF30A8003830F9
:10040000A90011270030A600F030A700FF30A80097
:100410003830A90011270030A600F230A700FF30C5
:10042000A8003830A90011270030A600F330A7003B
:10043000FF30A8003830A90011270030A600F330A3
:10044000A700FF30A8007830A90011270030A600CF
:10045000F730A700FF30A8007830A900112700303E
:10046000A600FF30A700A8007830A900112720308F
:10047000A600FF30A700A8007830A900112760303F
:10048000A600FF30A700A8007830A9001127E030AF
:10049000A600FF30A700A8007830A9001127F0308F
:1004A000A600FF30A700A8007830A9001127F2307D
:1004B000A600FF30A700A8007830A9001127F3306C
:1004C000A600FF30A700A8007830A9001127F3305C
:1004D000A600FF30A700A800F830A9001127F730C8
:1004E000A600FF30A700A800F830A9001127FF30B0
:1004F000A600A700A800F830A9001127FF30A60029
:10050000A700DF30A800F830A9001127FF30A600AF
:10051000A7009F30A800F830A9001127FF30A600DF
:10052000A7001F30A800F830A9001127FF30A6004F
:10053000A7000F30A800F830A9001127FF30A6004F
:10054000A7000D30A800F830A9001127FF30A60041
:10055000A7000C30A800F830A9001127FF30A60032
:10056000A7000C30A800D830A9001127FF30A60042
:10057000A7000830A800D830A9001127FF30A60036
:10058000A7000030A800D830A9001127FF30A6002E
:10059000DF30A7000030A800D830A9001127FF30B5
:1005A000A6009F30A7000030A800D830A90011276E
:1005B000FF30A6001F30A7000030A800D830A900E7
:1005C0001127FF30A6000F30A7000030A800D83058
:1005D000A9001127FF30A6000D30A7000030A800A9
:1005E000D830A9001127FF30A6000C30A70000303A
:1005F000A800D830A9001127FF30A6000C30A700B2
:100600000030A8009830A9001127FF30A60008305C
:10061000A7000030A8009830A9001127FF30A600DD
:100620000030A700A8009830A9001127DF30A600ED
:100630000030A700A8009830A90011279F30A6001D
:100640000030A700A8009830A90011271F30A6008D
:100650000030A700A8009830A90011270F30A6008D
:100660000030A700A8009830A90011270D30A6007F
:100670000030A700A8009830A90011270C30A60070
:100680000030A700A8009830A90011270C30A60060
:100690000030A700A8001830A90011270830A600D4
:1006A0000030A700A8001830A90011270800033067
:1006B000A600A700A800FB30A90011270330A60060
:1006C000A7001C30A800DB30A90011270330A600CA
:1006D000A700E030A800DB30A90011270330A600F6
:1006E0001C30A700E030A8009B30A9001127033080
:1006F000A600E030A700A8009B30A90011271C30FD
:10070000A600E030A700A8001B30A9001127E030A8
:10071000A600A700A8001B30A9001127E030A60002
:10072000A7001C30A8001B30A9001127E030A6004C
:10073000A7000330A8003B30A9001127E030A60035
:100740001C30A7000330A8003B30A9001127E0307F
:10075000A6000330A700A8007B30A90011271C3099
:10076000A6000330A700A8007B30A90011270800CD
:100770002030A6004030A7008030A8001B30A90020
:1007800011274030A6008030A7001030A8001B3091
:10079000A90011278030A6001030A7000230A80061
:1007A0001B30A90011271030A6000230A70001302D
:1007B000A8001B30A90011270230A6000130A700B5
:1007C0000030A8003B30A90011270130A6000030FE
:1007D000A7000430A8005B30A90011270030A60054
:1007E0000430A7002030A8009B30A9001127043056
:1007F000A6002030A7004030A8001B30A900112718
:10080000203008000030A600A7000830A8000F30F4
:10081000A90011270030A6000830A700A8000D305D
:10082000A90011270830A600A7000030A8000D304D
:10083000A90011270830A6000030A700A8000D303D
:10084000A90011270030A600A700A8000D30A900BC
:1008500011270830A6000030A700A8001C30A9000E
:1008600011270030A600A700A8001C30A9001127FE
:100870000830A6000030A700A8001B30A9001127EF
:10088000B830A6000030A700A8009B30A9001127AF
:100890005530A600B030A7000030A8005B30A9009A
:1008A00011271430A6005530A700B030A8003B3007
:1008B000A90011270030A6001630A7005530A80067
:1008C0001B30A90011270030A600A7001630A80091
:1008D0001B30A90011270030A600A700A8001B307C
:1008E000A900112708000030A600A700A800A90051
:1008F0001127FF30A600A700A800E030A9001127AB
:10090000FF30A600A700A800E830A9001127FF309B
:10091000A600A700A800F030A9001127FF30A6000C
:10092000A700A800F830A9001127FF30A600A700F3
:10093000A800F030A9001127FF30A600A700A800EA
:10094000E830A9001127FF30A600A700A800E0307A
:10095000A900112708000030A600A700A800FB305E
:10096000A90011270430A600A700A8001B30A90089
:1009700011272030A600A700A8001B30A9001127CE
:100980004030A600A700A8001B30A9001127803026
:10099000A600A700A8001B30A90011271030A60050
:1009A000A700A8001B30A90011270230A600A7004D
:1009B000A8001B30A90011270130A600A700A8003D
:1009C0001B30A90011270800FF30A6000030A70047
:1009D000A8009B30A9001127B630A6004930A70017
:1009E0000030A8009B30A90011270030A600B630C7
:1009F000A7004930A8005B30A90011270030A600ED
:100A0000A700FF30A8003B30A90011270030A60046
:100A10004930A700B630A8003B30A9001127493063
:100A2000A600B630A7000030A8005B30A90011274F
:100A300008000030A600A700FF30A8003B30A90046
:100A400011270030A6000830A700F730A8003B307F
:100A5000A90011270830A600F730A7000030A80031
:100A60005B30A9001127FF30A6000030A700A800C6
:100A70009B30A9001127F730A6000830A7000030EE
:100A8000A8009B30A90011270030A600F730A7006E
:100A90000830A8005B30A900112708004930A600E3
:100AA000A700A8001930A90011272430A60049305A
:100AB000A7009230A8009930A90011270030A600A5
:100AC000FF30A7000030A8005930A900112792304C
:100AD000A6004930A7002430A8003930A90011270A
:100AE00008009230A6000030A700A8001930A90025
:100AF0001127DB30A6000030A700A8001930A9009C
:100B000011276D30A6000030A700A8009930A90079
:100B100011272430A600A7000030A800D930A90072
:100B200011270030A6006D30A7000030A800593012
:100B3000A90011270030A600DB30A7000030A80074
:100B40001930A90011270030A6009230A700A80094
:100B50001930A90011270030A600A700DB30A8003B
:100B60001930A90011270030A600A7006D30A80099
:100B70003930A90011270030A6002430A700A800B2
:100B80007930A90011270030A6006D30A700003091
:100B9000A8005930A90011270030A600DB30A700BB
:100BA0000030A8001930A90011279230A600A70034
:100BB0000030A8001930A900112708000230A60053
:100BC0000030A700A8001930A90011270130A600A5
:100BD0000030A700A8001930A90011270030A60096
:100BE000A700A8009930A90011270430A600003002
:100BF000A700A8001930A90011272030A600003056
:100C0000A700A8001930A90011274030A600003025
:100C1000A700A8001930A90011278030A6000030D5
:100C2000A700A8001930A90011271030A600003035
:100C3000A700A8001930A90011270830A60000302D
:100C4000A700A8001930A90011270030A60008301D
:100C5000A7000030A8001930A90011270030A60015
:100C60000430A7000030A8001930A9001127003077
:100C7000A6002030A7000030A8001930A9001127D5
:100C80000030A6004030A7000030A8001930A900AD
:100C900011270030A6008030A7000030A8001930CE
:100CA000A90011270030A6001030A7000030A800CE
:100CB0001930A90011270030A6000230A70000302B
:100CC000A8001930A90011270030A6000130A700A4
:100CD0000030A8001930A90011270030A600A70095
:100CE000A8005930A90011270030A600A700A800CD
:100CF0003930A90011270030A600A7000430A80051
:100D00001930A90011270030A600A7002030A80044
:100D10001930A90011270030A600A7004030A80014
:100D20001930A90011270030A600A7008030A800C4
:100D30001930A90011270030A600A7001030A80024
:100D40001930A90011270030A600A7000230A80022
:100D50001930A90011270030A600A7000130A80013
:100D60001930A90011270030A600A7000830A800FC
:100D70001930A900112708000030A6000830A7008C
:100D80000030A8001B30A90011270830A600003051
:100D9000A700A8001B30A90011275D30A600003075
:100DA000A700A8001B30A9001127A230A6005530CB
:100DB000A7000030A8009B30A90011270030A60032
:100DC000A230A7005530A8005B30A90011270030E1
:100DD000A600A700F730A8003B30A900112700307B
:100DE000A600A700FF30A8003B30A9001127003063
:100DF000A600A7000830A8001B30A900112700306A
:100E0000A6000830A7000030A8001B30A900112759
:100E10000830A600A7000030A8001B30A900112749
:100E2000080029081839AA000310AA0C0310AA0CFC
:100E30000310AA0CAA0A29080739AB00AB0A031051
:100E4000AB0D0310AB0D0310AB0D0310AB0D031076
:100E5000AB0D860126088700A91B061686162A08F0
:100E6000532786122A08043C031D532786012708AE
:100E70008700291B061606172A08532706132A0877
:100E8000043C031D5327860128088700A91A06166B
:100E900086172A08532786132A08043C031D532764
:100EA000AB0B292F0800A2000130A1001D30A000CB
:100EB000A00B582FA10B562FA20B542F08008316FE
:100EC000003087008600031783129E019F010313E1
:100ED0002410A50173247324732473247324E4243D
:100EE000E424E424E424E4244E254E254E254E2516
:100EF0004E2571257125712571257125E720E72083
:100F0000E720E720E720DE25BC26DE25BC26DE25FF
:100F1000BC26012001200120012001200120012008
:100F20000120012001200120AB24AB24AB24AB2401
:100F3000AB24572357235723572357233E203E20C4
:100F40003E203E203E2002240224022402240224C9
:100F5000B823B823B823B823B82319251925192590
:100F6000192519259F219F219F219F219F219F2185
:020F70006A2FE6
:02400E00D430AC
:00000001FF
